:100000000C9493020C94CB020C94CB020C94CB0274
:100010000C94CB020C94CB020C94CB020C94CB022C
:100020000C94CB020C94CB020C94DC250C94AE26E1
:100030000C94BB200C94CB020C94CB020C94CB02FE
:100040000C94CB020C94CB020C94CB020C94CB02FC
:100050000C94CB020C9443210C94CB020C94CB0255
:100060000C94CB020C94CB020C94CB020C94CB02DC
:100070000C94CB020C94CB020C94CB020C94CB02CC
:100080000C94CB020C94CB020C94CB020C94CB02BC
:100090000C94CB020C94CB020C94CB020C94CB02AC
:1000A0000C94CB020C94CB020C94CB0282058205FB
:1000B000AE05AE05160634064C074C073F06D806BB
:1000C000E906E9061B2742273A2842273A288E27C5
:1000D000B1273A28082817282B0014001A00080016
:1000E000150017001C0018000C00120013002A0055
:1000F000E00004001600070009000A000B000D00D4
:100100000E000F003300340029001D001B00060004
:1001100019000500110010003600370038002800D3
:10012000C65CC75CE300E200E1002C002C0001513A
:100130005000510052004F0001001E001F0020001F
:1001400021002200230024002500260027000100B2
:1001500001003A003B003C003D003E003F002D0006
:100160002E002F003000310001004000410042000D
:1001700043004400450001004B004A00010001001B
:10018000CA5CCB5C005C460001000100010001007C
:100190004E004D0001004C0000047F3F1F643214EC
:1001A000643214783C1E1E140A05222325262829B1
:1001B0002A2C2D2F3032333536383A3B3D3E4042E3
:1001C000434547494A4C4E5051535557595A5C5E26
:1001D0006062646668696B6D6F71737577797B7D3A
:1001E0007F81838587898A8C8E90929496989A9C39
:1001F0009E9FA1A3A5A7A8AAACAEAFB1B3B4B6B851
:10020000B9BBBCBEBFC1C2C3C5C6C7C9CACBCCCDB2
:10021000CED0D1D2D2D3D4D5D6D7D7D8D9D9DADA8D
:10022000DBDBDBDCDCDCDCDCDDDDDDDDDCDCDCDC0D
:10023000DCDBDBDBDADAD9D9D8D7D7D6D5D4D3D241
:10024000D2D1D0CECDCCCBCAC9C7C6C5C3C2C1BF1F
:10025000BEBCBBB9B8B6B4B3B1AFAEACAAA8A7A583
:10026000A3A19F9E9C9A98969492908E8C8A89873F
:100270008583817F7D7B79777573716F6D6B69681D
:10028000666462605E5C5A5957555351504E4C4AF1
:100290004947454342403E3D3B3A3836353332309C
:1002A0002F2D2C2A292826252322FFAA7F554000FE
:1002B0000101010101010101010202020202020227
:1002C00002020303030303030303040404040404FA
:1002D00004050505050506060606060707070707C0
:1002E00008080808090909090A0A0A0B0B0B0C0C73
:1002F0000C0D0D0D0E0E0E0F0F0F1010111111120F
:100300001213131414151516161717181819191A8D
:100310001A1B1B1C1D1D1E1E1F20202122222324F0
:1003200024252626272829292A2B2C2D2D2E2F302F
:10033000313232333435363738393A3B3C3D3E3F43
:10034000404142434445464748494A4C4D4E4F5030
:10035000515354555658595A5B5D5E5F61626465EE
:100360006668696B6C6D6F7072737577787A7B7D78
:100370007E8082838587888A8C8E8F9193959698CC
:100380009A9C9EA0A2A3A5A7A9ABADAFB1B3B5B7E8
:10039000BABCBEC0C2C4C6C9CBCDCFD1D4D6D8DBBF
:1003A000DDDFE2E4E7E9EBEEF0F3F5F8FAFDFF0C50
:1003B000035A006C0061006E007400000020034DC1
:1003C000006100740074006800650077002000433D
:1003D000006F007200640069006500720000000494
:1003E00003090409023B00020100A0FA090400000D
:1003F000010301010009211101000122400007054C
:100400008103080001090401000103000000092123
:100410001101000122B6000705820320000112012C
:10042000000200000008EDFE606001000102000112
:1004300005010902A10185020901A10005091901AF
:10044000290815002501950875018102050109306B
:1004500009311581257F95027508810609381581B6
:10046000257F950175088106050C0A38021581253E
:100470007F950175088106C0C005010980A101852D
:100480000319012AB700150126B7009501751081DF
:1004900000C0050C0901A101850419012AA002155B
:1004A0000126A002950175108100C005010906A171
:1004B000018506050719E029E7150025019508754E
:1004C0000181020507190029EF1500250195F07536
:1004D000018102050819012905950575019102950B
:1004E0000175039101C005010906A101050719E085
:1004F00029E7150025019508750181029501750808
:1005000081010507190029FF150026FF00950675D2
:1005100008810005081901290595057501910295C5
:100520000175039101C011241FBECFEFDAE0DEBFD9
:10053000CDBF04B603FE18C080911403909115033B
:10054000A0911603B09117038730904BA740B04B92
:1005500059F410921403109215031092160310927E
:100560001703E0E0F8E3099511E0A0E0B1E0EAED5F
:10057000F2E502C005900D92A43CB107D9F723E043
:10058000A4ECB1E001C01D92A431B207E1F70E94D2
:1005900058130C946B290C94000081E0089581E0BD
:1005A00008950C94CF0208950C94D3021F93CF9317
:1005B000DF9300D000D01F92CDB7DEB749835A83B6
:1005C0006B833091C70189819A81311114C06623F0
:1005D00059F0222349F00E948909182F682F898138
:1005E0009A810E94320903C00E945D09182F698117
:1005F0007A81812F04C00E94890969817A810F90D4
:100600000F900F900F900F90DF91CF911F910C944E
:10061000C310FC01262F4081518162817381848146
:100620000C94D60281E00895CF93DF93EC0160E053
:100630000E940903BE01DF91CF910C94D4020C9467
:1006400009120C94051208950E94DC070E942303EE
:100650002FEF84E39CE0215080409040E1F700C000
:1006600000000C9469210F931F93CF93DF938C01AB
:1006700061E00E940903EC01B8010E94D1028823C5
:1006800009F444C0B801CE010E94061F8823F1F18D
:10069000B801CE010E941A1D8823C1F1B801CE0114
:1006A0000E94621E882391F1B801CE010E94201C95
:1006B000882361F1F8018281882309F1CB358DE52A
:1006C000D807C1F050F4C115FCE5DF0781F0CF3D3C
:1006D000DC45A9F40E94C00E19C0CC35EDE5DE075B
:1006E00061F0CD35DD4559F40E94030E08C00E942B
:1006F00024030CC00E940C0E02C00E940F0EC80101
:10070000DF91CF911F910F910C94CD0280E0DF918A
:10071000CF911F910F9108950E949D200C94A503E5
:100720000E94A8030C94A32008950C94940381E0E4
:1007300008950C9497030895CF93C82F0E949503B2
:100740008C2F0E949903CF91089580E00C949C0314
:100750000E94621F0C949C030E94621F9091C6012C
:10076000891721F08093C6010C949C030895CF93C0
:10077000DF93CDB7DEB72B970FB6F894DEBF0FBE71
:10078000CDBF4F83588769877A878B8761110E9415
:100790004F0D9E012F5F3F4F86E0F90111928A9520
:1007A000E9F785E0FE013796D90101900D928A950F
:1007B000E1F789819A814C815D81452B31F09F3F22
:1007C00031F491E08F3F19F403C091E001C090E053
:1007D00090FF09C049815A816B817C818D819E8106
:1007E0000E94700C05C0C9010E9412038111F2CF52
:1007F0002B960FB6F894DEBF0FBECDBFDF91CF9121
:100800000895FC01808191810E94CB090895CF93C6
:10081000882309F4A4C0C82F8238C1F40E94621F43
:1008200081FD9DC069E380910201909103010E94C6
:1008300058200E94710D2FEF81EE94E021508040EE
:100840009040E1F700C0000069E319C0833801F56A
:100850000E94621F80FD83C063E580910201909138
:1008600003010E9458200E94710D2FEF81EE94E049
:10087000215080409040E1F700C0000063E5809186
:100880000201909103010E946320CF910C94710D9D
:100890008438C1F40E94621F82FD61C067E48091C8
:1008A0000201909103010E9458200E94710D2FEFC8
:1008B00081EE94E0215080409040E1F700C00000BC
:1008C00067E4DDCF8CEF8C0F813AD0F46C2F8091F0
:1008D0000201909103010E94D81F882349F06C2FD8
:1008E00080910201909103010E9463200E94710D8A
:1008F0006C2F80910201909103010E945820C5CF76
:1009000080E28C0F883048F4C77081E001C0880F06
:10091000CA95EAF70E94320DB8CFEBE5EC0FE33051
:1009200040F4F0E0E65AFE4F808190E0CF910C94C5
:10093000961FE8E5EC0FE73150F4F0E0EE0FFF1FF3
:10094000E45DFE4F80819181CF910C94AC1FCD3E30
:1009500030F08C2F0E94DD13CF910C94AF14CF9107
:100960000895882309F464C0823879F40E94621FD4
:1009700081FF5EC069E380910201909103010E94B2
:1009800058200E94710D69E310C08338B1F40E94B1
:10099000621F80FF4DC063E58091020190910301C9
:1009A0000E9458200E94710D63E580910201909190
:1009B00003010E9463200C94710D843879F40E9425
:1009C000621F82FF35C067E48091020190910301AC
:1009D0000E9458200E94710D67E4E7CF9CEF980FAA
:1009E000913A10F4682FE1CF90E2980F983050F4CC
:1009F000877091E001C0990F8A95EAF7892F0E94CC
:100A0000380DD9CF9BE5980F933020F480E090E02B
:100A10000C94961F98E5980F973120F480E090E0B1
:100A20000C94AC1F8D3E20F00E9438140C94AF142F
:100A300008951F93CF93DF93182FEB010E940704B3
:100A4000209741F08FE99FE00197F1F700C0000087
:100A50002197F6CF812FDF91CF911F910C94B10494
:100A6000893319F060E070E002C060E570E00C943A
:100A70001905882321F00E94320D0C94710D089500
:100A8000882321F00E94380D0C94710D0895CF92A7
:100A9000DF92EF92FF920F931F93CF93DF937C012E
:100AA000D62FC72FFC011281058102950F700E947D
:100AB000280D8823B9F01123A9F08C2F807F803472
:100AC00021F080E28D0F883068F08091C90282FDAC
:100AD00009C082E00E94D10D0E94280D91E0D82E1D
:100AE000D92601C0D12CCC2EC2948FE0C8228C2DE7
:100AF00090E08C30910508F0CFC1FC01EA5AFF4F1D
:100B00000C94C6288C2F807FCF70882311F0C2955B
:100B1000C07F112399F0CC2309F4AAC180E28D0F84
:100B2000883010F0D11104C08C2F0E94320D03C008
:100B30008C2F0E94420D0E94710D9AC18D2F0E9430
:100B4000B104CC2309F4A8C180E28D0F883038F1BC
:100B5000DD2329F18C2F0E94480D24C08C2F807F2B
:100B6000CF70803211F0C295C07FDD2319F0D130F3
:100B7000A1F13DC08091C90282FF17C0112349F045
:100B8000CC2329F08C2F0E94320D0E94710D80E041
:100B900070C180E00E94B104CC2309F47DC18C2F88
:100BA0000E94380D0E94710D77C1112371F000234E
:100BB00041F0013031F40E94520D8C2B0E945A0DED
:100BC0006BC10E94520D8C2B1DC0002319F0013007
:100BD00009F462C10E94670D25C0112321F006307F
:100BE00008F05AC10EC0053008F056C11BC01123D1
:100BF00061F0002331F0F701858180FF39C18F70EA
:100C000085838C2F0E94390547C1002359F0D933C1
:100C100009F03FC1FFEF07EE13E0F1500040104034
:100C2000E1F735C18C2F0E94400536C18C2F869587
:100C30008695837019F0813061F02EC1112321F067
:100C40008D2F9C2F937002C080E090E00E94961F31
:100C50002BC1112321F08D2F9C2F937002C080E0B7
:100C600090E00E94AC1F20C18D2F112319F00E942B
:100C7000DD1302C00E9438140E94AF1415C18C2FDE
:100C8000837009F047C011110BC12D2F22952695B5
:100C90002770220F220F6D2F6F70862F90E0A0E03B
:100CA000B0E0022E04C0880F991FAA1FBB1F0A9430
:100CB000D2F7D4FF10C04FE050E060E070E004C015
:100CC000440F551F661F771F2A95D2F74095509500
:100CD0006095709503C040E050E0BA01C695C69596
:100CE000C3708A019B01082B192B2A2B3B2BC901AE
:100CF000B801C23049F058F4C13019F00E944808D8
:100D0000CFC00E943608CCC00E945A08C9C00E94B9
:100D10003408C6C0112319F08C2F817001C086954C
:100D2000882309F4BDC02D2F229526952770220F08
:100D3000220F6D2F6F70862F90E0A0E0B0E0022EA2
:100D400004C0880F991FAA1FBB1F0A94D2F7D4FFB3
:100D500010C04FE050E060E070E004C0440F551F49
:100D6000661F771F2A95D2F740955095609570952C
:100D700003C040E050E0BA01C695C695C3708A0131
:100D80009B01082B192B2A2B3B2BC901B801C23020
:100D900049F058F4C13019F00E940D0981C00E9439
:100DA000FB087EC00E941F097BC00E946E0878C0AD
:100DB000CF70112339F08C2F0E9494088D2F0E9440
:100DC00039056EC08D2F0E9440058C2F0E94B508FA
:100DD00067C0D23F21F128F4D03F41F0D13FC1F0AC
:100DE00043C0D33F19F1D43F79F03EC0112341F005
:100DF000053008F051C08C2F8F710E94DA084CC06A
:100E0000063008F049C0F7CF8091C90282FF18C0B0
:100E1000112339F08C2F8F710E9494083DC011234B
:100E2000C9F38C2F8F710E94B50836C0112329F0A9
:100E30008C2F8F710E947F082FC00E947A082CC0CF
:100E4000112349F0CF718C2F0E94940863E08C2FFE
:100E50000E94B60D21C081E00E94D10D0230E0F069
:100E600082E00E94D10D18C0112331F0002391F2CD
:100E70008D2F0E94070410C0002399F2D93349F442
:100E80001FEF27EE33E0115020403040E1F700C063
:100E900000008D2F0E94B10488EF8C0D843020F467
:100EA0000E94621F0E949C03DD20C9F00E94240D55
:100EB00080FD15C0F70112820E941E0D0E94940849
:100EC000C7010E9490070E941E0DDF91CF911F91D4
:100ED0000F91FF90EF90DF90CF900C94B508DF91C9
:100EE000CF911F910F91FF90EF90DF90CF900895D9
:100EF0000F931F93CF93DF93EC01688179818A81EF
:100F00000E94D6098C010E9431090E942208B80172
:100F1000CE010E944705DF91CF911F910F91089557
:100F2000CF93DF93EC01988189812B813C81232B26
:100F300031F08F3F31F481E09F3F19F403C081E02D
:100F400001C080E080FD1DC0CE010E9433038111ED
:100F500010C00E94280D8823A1F08A81882389F07F
:100F60008091C90282FD0DC082E0DF91CF910C9487
:100F7000D10DCE010E947807CE01DF91CF910C9464
:100F80001403DF91CF91089580E090E00E94961FB6
:100F900080E090E00E94AC1F0E944F0D0E94710DF6
:100FA0000E94E0150C94AF1480910201909103010E
:100FB0000E946E200C94C4070E943F0D0C94D4072D
:100FC00092959F70963079F010F4925001C09A502B
:100FD000923068F4803F69F018F4883E40F409C00C
:100FE000843F29F406C0883E20F0813F11F080E064
:100FF000089581E00895FC01808191810E94CB09D0
:101000000E94E0070895CF93DF9300D000D01F9295
:10101000CDB7DEB70F900F900F900F900F90DF912C
:10102000CF910895CF93DF9300D000D000D0CDB7FB
:10103000DEB726960FB6F894DEBF0FBECDBFDF91A8
:10104000CF910895089508950C9423080C942408D2
:101050000E9426086093EA017093EB018093EC01F3
:101060009093ED010C94C4070C9428080F931F93E0
:101070000091EA011091EB012091EC013091ED011A
:10108000602B712B822B932B1F910F910C942808AE
:101090000F931F930091EA011091EB012091EC0155
:1010A0003091ED0160237123822393231F910F91CF
:1010B0000C9428080F931F930091EA011091EB0103
:1010C0002091EC013091ED01602771278227932751
:1010D0001F910F910C9428080C9423080E946C080F
:1010E0006093E6017093E7018093E8019093E90132
:1010F0000C94C40760E070E0CB010C946E080F9371
:101100001F9341E050E060E070E08A019B0104C061
:10111000000F111F221F331F8A95D2F7C901B80192
:101120001F910F910C946E080F931F9341E050E0B4
:1011300060E070E004C0440F551F661F771F8A955A
:10114000D2F78091E6019091E701A091E801B0917A
:10115000E9018A019B01082B192B2A2B3B2BC90182
:10116000B8011F910F910C946E080F931F9341E0EB
:1011700050E060E070E004C0440F551F661F771F09
:101180008A95D2F740955095609570958091E601CB
:101190009091E701A091E801B091E9018A019B01DA
:1011A000082319232A233B23C901B8011F910F915A
:1011B0000C946E080F931F9341E050E060E070E0E4
:1011C00004C0440F551F661F771F8A95D2F7809180
:1011D000E6019091E701A091E801B091E9018A014F
:1011E0009B01082719272A273B27C901B8011F910E
:1011F0000F910C946E080F931F930091E6011091CC
:10120000E7012091E8013091E901602B712B822BDD
:10121000932B1F910F910C946E080F931F930091C5
:10122000E6011091E7012091E8013091E901602386
:101230007123822393231F910F910C946E080F93B7
:101240001F930091E6011091E7012091E801309190
:10125000E90160277127822793271F910F910C9432
:101260006E0808952CE0929F800D1124E82FE695DA
:10127000E695E695877051E001C0550F8A95EAF72B
:1012800085E0E89FF0011124E853FE4F20E030E0B4
:1012900070E04081CB01022E02C0969587950A949A
:1012A000E2F78170819584278523842781932F5FBE
:1012B0003F4F2530310569F708952CE0929F800D4E
:1012C0001124682F669566956695982F977085E02E
:1012D000689FB001112440E050E080E0FB01E40F82
:1012E000F51FE853FE4F208130E0092E02C03695ED
:1012F00027950A94E2F721703327042E01C0220FAC
:101300000A94EAF7822B4F5F5F4F4530510531F762
:101310000895BF92CF92DF92EF92FF920F931F93A7
:10132000CF93DF938C01C090E601D090E701E0906D
:10133000E801F090E9018091EA019091EB01A09120
:10134000EC01B091ED01C82AD92AEA2AFB2ACFE1A3
:10135000D0E0D701C6010C2E04C0B695A79597958D
:1013600087950A94D2F780FD04C0219790F7B12C9D
:1013700007C0BC2EB8018C2F0E94D6100197A9F38C
:101380008B2DDF91CF911F910F91FF90EF90DF9008
:10139000CF90BF900895CF93DF93EC010E9489090D
:1013A000BE010E94D610DF91CF9108951F93CF9375
:1013B000DF93EB019091C701992321F0CB010E94AB
:1013C000CB0913C0882349F0CB010E948909182F4B
:1013D000682FCE010E94320904C0CB010E945D0932
:1013E000182FBE01812F0E94D610DF91CF911F913F
:1013F00008951F93CF93DF93C091EE0116E0809183
:10140000EF01C81799F0D0E01C9FF0011D9FF00D6F
:101410001124E051FE4F40815181628173818481AA
:1014200095810E9412082196C770E9CFDF91CF9174
:101430001F91089540912002509121026091220253
:101440007091230280912402909125020C9412083D
:10145000EF92FF920F931F93CF93DF93809125021A
:1014600082958F7009F065C080912202882309F46B
:1014700060C08091EE01F090EF0110912002009188
:101480002102609123027091240291E01F3F09F034
:1014900090E0C0910001D0910101292F96E0E92E42
:1014A0008F1509F446C06115710521F00F3F21F039
:1014B00030E003C031E001C0322F90E030FD36C093
:1014C000E89EF001E99EF00D1124DF01A051BE4F0E
:1014D00011963C911197301329C03C91311326C0CD
:1014E00012963C911297311121C013964D915C9147
:1014F0001497461B570B4C175D07C0F480912502CB
:101500008F70806180932502EB50FE4F80818F7039
:101510008061808380E292E00E949007DF91CF910A
:101520001F910F91FF90EF900C94F909019687702D
:10153000B7CFDF91CF911F910F91FF90EF9008955A
:101540009F92AF92BF92CF92DF92EF92FF920F9352
:101550001F93CF93DF93CDB7DEB761970FB6F894A3
:10156000DEBF0FBECDBF8C0185E0F801DE011D9608
:1015700001900D928A95E1F7D8011296EC90909126
:101580002002E091210220912302309124022115B2
:10159000310531F0EF3F31F481E09F3F19F403C092
:1015A00081E001C080E0B82FB1709B2E80FD47C163
:1015B000D8014C9111965C9111971396AD90BC9007
:1015C000149780E2C82E82E0D82EF0902202B50156
:1015D000621B730B2091000130910101FF2009F47F
:1015E000D9C0809125026217730708F095C0282F93
:1015F000207F09F052C05E1313C0491311C0FE2CA6
:10160000E1100EC08F708061809325020E941A0A3B
:10161000C6010E94900780912502F80185834DC183
:10162000AB2831F05F3F31F481E04F3F19F403C044
:1016300081E001C080E080FD03C081E08E2502C012
:1016400080E090E0F82FF170FF2E80FF1CC08091A9
:10165000EE012091EF0136E0821709F40BC190E012
:10166000389FF001399FF00D1124E051FE4F618148
:10167000561306C06081461303C06281E61203C0A0
:1016800001968770E9CFFE2CEE2009F416C18091F7
:10169000250281608093250254C05E1306C0491361
:1016A00004C0E11002C0F80199C0C8010E94FB0704
:1016B000882361F1EE2051F120912502822F82953D
:1016C0008F7090E0029774F0809120029091210237
:1016D00098878F831986BB86AA862C87CE010796AA
:1016E0000E94900786E0F801A0E2B2E001900D921E
:1016F0008A95E1F70E94280A0E941A0A0AC05E171A
:1017000011F1C8010E94FB0781112CC0C8010E9481
:101710009007FF24F394D1C0282F207F81F77A2DE2
:10172000B98AA88A6E2D89890E94030880E292E016
:101730000E94900786E0D6011D928A95E9F70E94E3
:101740001A0AF12CBAC04913DCCFE110DACFF80144
:101750008583C8010E94900786E0D6011D928A9574
:10176000E9F7ABC0EE2091F220912502822F8295FD
:101770008F7090E002970CF4B5CF80912002909189
:1017800021029A8389831B82BD82AC822E83CE0183
:101790000196A6CF6217730708F044C0FE2CEE2016
:1017A00009F4B4CF5E1330C049132EC02091250236
:1017B00020FD21C0822F82958F70482F50E0411567
:1017C0005105C9F0F80125834F30510541F08F5F75
:1017D000982F9295907F822F8F70892B8583C801D7
:1017E0000E94900786E0F801A0E2B2E001900D921D
:1017F0008A95E1F73CC086E0F801A0E2B2E00190F2
:101800000D928A95E1F759C0C8010E94FB0781112A
:1018100069CF80912502816080932502C8010E94D2
:1018200090074BC07A2DB98AA88A6E2D89890E94AB
:10183000030886E0D6011D928A95E9F718C0EE20CC
:1018400009F464CFC8010E94FB07F82E882309F42D
:101850005DCF86E0F801A0E2B2E001900D928A959A
:10186000E1F780E292E00E9401040E94280A0E94AF
:101870001A0A23C04D875E878D859E850E94CB09FD
:10188000292F22952F70223028F49F7039F0811172
:1018900005C00BC0243028F49F7049F4805E883066
:1018A00020F0C8010E9490079F2CF92C06C0D80197
:1018B00015969C91907F91F7F8CF8F2D61960FB67A
:1018C000F894DEBF0FBECDBFDF91CF911F910F9176
:1018D000FF90EF90DF90CF90BF90AF909F900895D2
:1018E0001F93CF93DF93CDB7DEB72C970FB6F89445
:1018F000DEBF0FBECDBF4F83588769877A878B873E
:101900009C87CE0107960E94A00A8823D1F09F8170
:1019100088852A853B85232B31F08F3F31F481E088
:101920009F3F19F403C081E001C080E080FD47C003
:101930004F81588569857A858B859C850E94120820
:101940003EC086E0FE013796DE01119601900D92B1
:101950008A95E1F7FF81E8856A857B8561157105C8
:1019600031F0EF3F31F481E0FF3F19F403C081E033
:1019700001C080E080FD23C02091EF0130E0C9016B
:101980000196877099274091EE0150E084179507E2
:10199000F1F1F983EA837D836C8396E0929FD00115
:1019A000939FB00D1124A051BE4FFE0131960190BE
:1019B0000D929A95E1F78093EF010E94F90916E0E4
:1019C0008091EE019091EF01891771F1189FC0018C
:1019D000112480519E4F0E94A00A882329F1E09192
:1019E000EE011E9FF0011124E051FE4F4081518114
:1019F00062817381848195810E9412088091EE0139
:101A000090E00196877099278093EE01D9CF0E94CC
:101A1000DC071092EF011092EE01E0E2F2E086E0C6
:101A2000DF011D928A95E9F72C960FB6F894DEBF78
:101A30000FBECDBFDF91CF911F91089580914602D7
:101A400085958595859508958091460287700895BE
:101A500090914602977081E009F480E008958091AA
:101A60006902089590916902892B80936902089513
:101A7000809590916902892380936902089510925C
:101A80006902089590916802892B809368020895F5
:101A9000809590916802892380936802089510923E
:101AA0006802089580914702089508950C94550D99
:101AB0000C94560D9091C90292FD08C09091470276
:101AC000981721F0809347020C94580D0895809147
:101AD0004702882329F01092470280E00C94580DA9
:101AE0000895CF93DF93E0910201F091030180917B
:101AF00069028083E0910201F0910301908180915D
:101B00006802892B808380914702882381F0E091CD
:101B10000201F09103019081892B80838091020161
:101B2000909103010E94C21F81110E94670DC09114
:101B30000201D091030140E250E066E272E0CE0182
:101B40000E941629892B69F080E2FE01A6E2B2E02C
:101B500001900D928A95E1F7CE01DF91CF910C941F
:101B60006E1FDF91CF9108950C94550D9091C9028D
:101B700092FD10C098E0899F90011124262B20939C
:101B800046020E9494088091460285958595859528
:101B90000C94B40D0C9494081092460280E00C94BE
:101BA000B40D209146028095822380934602982F9F
:101BB000977099F430E0482F082E000C550B24172D
:101BC000350759F09091C90292FD07C0859585951A
:101BD00085950E94B5080C94CC0D08959091C9028A
:101BE00092FB222720F9281769F080FB92F9909345
:101BF000C9028091C8029091C9020E943C0E82E005
:101C00000C94D10D08958091C90282FB882780F938
:101C100091E089270C94EE0D81E00C94EE0D80E0AC
:101C20000C94EE0D6FEF7FEF80E090E00C9455295F
:101C300080E090E00E94312921E0893E9E4F09F02A
:101C400020E0822F089582E090E00C94232983E025
:101C500090E00C942329CF9384E090E00E94232904
:101C6000C82F82E290E00E9423292C2F30E0A901A6
:101C7000582BCA01CF910895CF93C92F682F84E0C4
:101C800090E00E9437296C2F82E290E0CF910C9473
:101C90003729AB01BC018FE090E00C944929AB01DE
:101CA000BC0183E190E00C94492960E070E0CB0135
:101CB0000C944F0E60E070E0CB010E94490E0C9432
:101CC000550E69EE7EEF80E090E00E94552960E0BD
:101CD00082E090E00E94372960E083E090E00E947B
:101CE00037291092EA011092EB011092EC01109248
:101CF000ED0160E084E090E00E94372960E082E23C
:101D000090E00E94372960E085E090E00E9437294A
:101D100060E086E090E00E9437296FEF87E090E076
:101D20000E94372940E050E0BA0188E090E00E942C
:101D3000492960E08DE090E00E94372940E050E0C2
:101D4000BA0188E190E00E94492960E087E190E0D3
:101D50000E94372940E050E0BA018CE190E00E94F7
:101D6000492960E070E080E290E00E94552940E05F
:101D700050E0BA0188E190E00E9449290C945A0E83
:101D80000C94610E682F8EE090E00C9437290E942D
:101D90002821609376027093770280937802909363
:101DA000790260937202709373028093740290932D
:101DB0007502089585B7806885BF85B7806885BF3F
:101DC000089581E008950C94E10E08950C94E50EB9
:101DD0000C94E50E0C94E80E0C94E50E0C94EC0EAD
:101DE0000C94E50E0E94DA0E82EB91E10E94581FDE
:101DF0000E94F00E0C94EE0E0E94E60E0C94E50E7E
:101E00000E94CC110C949B030E9413210E94B112DA
:101E10000E94000F0E943F1B0C94EA0E5F926F928B
:101E20007F928F929F92AF92BF92CF92DF92EF926A
:101E3000FF920F931F93CF93DF93CDB7DEB72A970F
:101E40000FB6F894DEBF0FBECDBF0E94C612C82EDB
:101E500081110E94C70E3AE6832E32E0932E00E0F5
:101E600010E0502E802F0E94F0115C01F40161906F
:101E700071904F016826792661147104B1F40F5FE7
:101E80001F4F0430110569F78FEF89838A831B8206
:101E90000E941C218160782F9D838C8349815A8107
:101EA0006B818D810E94B7033AC080917A0281FDD7
:101EB0000E94F911D12CEE24E394F12CC3018E2160
:101EC0009F21892B29F10E94E30E8823A9F0DE824D
:101ED0005F82AE20BF2081E0AB2809F480E08887D4
:101EE0000E941C218160782F9A8789874E815F81AB
:101EF00068858A850E94B703000F111FF801E65913
:101F0000FD4F80819181E826F926F182E08207C0A9
:101F1000D394EE0CFF1CFCE0DF12D0CFB0CF81E0F9
:101F2000C11001C080E02A960FB6F894DEBF0FBE44
:101F3000CDBFDF91CF911F910F91FF90EF90DF9078
:101F4000CF90BF90AF909F908F907F906F905F9059
:101F500008950E940E0F0E94721B0E94CD140C94D3
:101F6000AC03CF93DF930E94DB10EC01811521E5D8
:101F7000920708F045C0811530E5930708F094C03A
:101F8000883E910528F5803E910508F0F8C0883A12
:101F9000910570F4853A910508F07CC08130910577
:101FA00009F475C008F4E8C0049708F0E8C0E4C07C
:101FB0008F3B910508F0E0C0C85AD0E0CC0FDD1F80
:101FC000C35ADE4F0990D881C02DCE019464D8C089
:101FD000811540E2940758F4811551E0950708F007
:101FE000CEC08D3E910508F4C7C09065C9C0C1152B
:101FF00080E4D80708F4C0C0DF70CE01906AC0C08A
:10200000811525E59207A8F4811534E5930708F0BA
:1020100095C0811543E5940708F07BC0811552E512
:10202000950708F061C0D82FCC27CE01816F906A48
:10203000A7C0C11589E5D807A0F4C11528E5D207C6
:1020400008F082C0C11536E5D30708F095C08C2F83
:102050000E946F118F7190E0D82FCC27CE01906233
:102060008FC0C1154AE5D40708F474C0CE0190565C
:102070008115904208F080C08D2F8F710E946F11E2
:10208000DD27D0628F71AE01582BCA0179C081E083
:1020900090E076C0C55AD0E0C557DE4F8881C82F82
:1020A000D0E0CE0190646CC074E0969587957A95E7
:1020B000E1F7282F23703C2F337081E090E002C0BD
:1020C000880F991F3A95E2F79C68AC01522B9A0150
:1020D0009C2F9F709695969550E2959FE001112454
:1020E000C9018C2B9D2B4CC08370992721E030E0D7
:1020F00002C0220F331F8A95E2F79C2F9695969582
:1021000080E2989FE0011124C22BD32BCE019C6862
:1021100037C08370992721E030E002C0220F331FBF
:102120008A95E2F79C2F9695969540E2949FE00160
:102130001124C22BD32BCE019A6822C0D82FCC27D2
:10214000CE01846F906A1CC0DC2FCC27CE01806F3B
:10215000906A16C08C2F8F700E946F1194E0D695F4
:10216000C7959A95E1F7CF70D0E0DC2FCC27D069E6
:102170009E01282BC90104C080E090E001C0CE017F
:10218000DF91CF91089520E3829FC0011124FC01CB
:102190002CE0729FE00DF11D1124E60FF11DEE0FF2
:1021A000FF1FE852FF4F8591949108950E94C3103C
:1021B0000E94B10F08958238910569F1B0F481331E
:1021C000910509F46DC048F48932910509F463C0A2
:1021D0008A32910509F469C008958533910509F49F
:1021E00055C089339105B9F00895833E910569F191
:1021F00038F4803E9105B1F0823E910509F10895D1
:10220000863E9105A9F1873E9105B9F1843E91057D
:1022100009F064C023C02091C80220FD4FC021FDF9
:102220004DC008958091C80280FD44C08091C902CC
:1022300080FF44C08091C80284FD42C083EE4DC03F
:102240008091C80282FF38C0F5CF8091C80282FD1C
:1022500033C08091C90280FD31C0ECCF8091C902AA
:1022600081FF32C08091C80284FD2AC087EE35C04C
:102270008091C80283FF26C0F5CF8091C80283FDFC
:1022800021C08091C90281FD1FC0ECCF8091C8029E
:1022900085FD1CC01DC08091C80285FD19C016C0F7
:1022A0008091C80286FD16C017C08091C80286FDC5
:1022B00013C010C089E311C082EE0FC080EE0DC0C4
:1022C00080E00BC086EE09C084EE07C089E205C03D
:1022D00085E303C08AE201C081E390E00895909114
:1022E000C80292FF0DC0282F2871283019F4877F6B
:1022F000846006C0282F2471243011F48B7F8860FD
:1023000093FF0DC0282F2871283119F4877E84612E
:1023100006C0282F2471243111F48B7E886120910E
:10232000C90220FF0DC0382F3871383019F4877F6B
:10233000816006C0382F3171313011F48E7F886092
:1023400021FF0DC0282F2871283119F4877E816163
:1023500006C0282F2171213111F48E7E886194FDF1
:10236000877E089580E008950C94120E0E94C61294
:102370008FE39CE90197F1F700C000000E94C612AC
:1023800080E00E94F01180FF04C00E94B4110C9400
:10239000692108950C94B6110E94180E811102C093
:1023A0000E94C00E0E94230E80937A020E942B0E80
:1023B0009093C9028093C8020E94CA110E94270EFE
:1023C000682F70E080E090E00E9434086091E601A0
:1023D0007091E7018091E8019091E9010C946C08FB
:1023E000E82FF0E0EE0FFF1FEE52FD4F808191814C
:1023F0000895089580EA8A95F1F7089500C0089538
:102400000C94FA1108950C9402120C9403120C947B
:1024100002120C940712F894E82FE295EF70F0E0A6
:1024200031A1282F2F7081E090E001C0880F2A95FC
:10243000EAF7982F9095932391A392A1892B82A3D9
:10244000789408950F931F93CF93DF93CAE9D1E057
:1024500089918F3F11F00E940B1281E0CE39D8078D
:10246000B9F7CEE8D1E00AE911E089918F3F11F088
:102470000E940B120C171D07C1F7DF91CF911F911E
:102480000F910895BF92CF92DF92EF92FF920F9338
:102490001F93CF93DF938C01C62FD0E0CE018656D9
:1024A0009E4F6C01FC0190819F3F09F450C0B62EF5
:1024B000F894E92FE295EF70F0E081A19F7021E0A0
:1024C00030E001C0220F9A95EAF7822B81A382A106
:1024D0002095282322A378940E94FE11EEE8F1E0D3
:1024E0004AE951E021E030E0E12CF12C61916F3FAD
:1024F00089F0A62FA295AF70B0E090968C9190E0F5
:102500006F7002C0959587956A95E2F780FD02C0CD
:10251000C90102C080E090E0E82AF92A220F331FA7
:102520004E175F0719F7F60180818F3F11F00E9467
:102530000B1261E0E114F10409F460E08B2D0E94BC
:102540000012CC0FDD1FC00FD11FF982E882DF918E
:10255000CF911F910F91FF90EF90DF90CF90BF90A0
:1025600008950E94221288E0E2EDF2E0DF01982F48
:102570001D929A95E9F7EAECF2E0DF011D928A9547
:10258000E9F784E00E9411130C941F03FF920F934C
:102590001F93CF93DF93CDB7DEB728970FB6F8948C
:1025A000DEBF0FBECDBF8E010F5F1F4F88E0F80169
:1025B00011928A95E9F7F12C6F2DC8010E94421201
:1025C000F394F4E0FF12F8CF48E050E0B8018AEC51
:1025D00092E00E941629FF24F394009709F4F12C4D
:1025E000892B41F088E0F801AAECB2E001900D924D
:1025F0008A95E1F72F2D44E062ED72E08AEC92E0DB
:102600000E9412130E9421038F2D28960FB6F89472
:10261000DEBF0FBECDBFDF91CF911F910F91FF9015
:1026200008950895FF920F931F93CF93DF93F82E91
:10263000092F162FD72FC42F222349F081E0809332
:102640007D020E941C2190937C0280937B028091EA
:102650007D028823D9F080917B0290917C020E94B8
:102660003421059798F0EF2DF02FA12FBD2F80E09A
:1026700090E04C2F50E08417950734F4219131916C
:102680002D933D930196F7CF10927D02DF91CF916C
:102690001F910F91FF9008950E9434230E94040F10
:1026A0000C9440230E9444230E94A90F0C945E23A3
:1026B0000E94BA200E941B230E94F20E0E944C131B
:1026C0000E9452130E94FC0EFBCF8091840280FF77
:1026D00006C06091090170E0660F771F26C081FF78
:1026E00004C06091090184E005C082FF07C06091C9
:1026F000090188E0689FB001112417C090918302FE
:102700009923D1F060910801961788F7209109016B
:1027100088E0289F90011124929FA001939F500D63
:10272000112470E0CA010E9490286038710540F4BD
:102730006115710519F406C068E070E0862F0895F0
:102740008FE7089581E008958091840280FF08C09A
:102750006091050170E0759567957595679521C045
:1027600081FF06C06091050170E07595679519C0FD
:1027700082FF04C06091050170E010C09091820258
:10278000992399F0609104019617A0F780910501B3
:10279000899FC001112470E00E9490286038710563
:1027A00040F46115710519F406C061E070E0862FF0
:1027B00008958FE7089581E008958D3E21F40E94E9
:1027C0006513819504C08E3E29F40E9465138093A1
:1027D000880208958F3E21F40E946513819504C0FC
:1027E000803F29F40E946513809387020895893FF2
:1027F00019F40E94A41305C08A3F31F40E94A41367
:1028000081958093890208958B3F21F40E94A4133F
:10281000819504C08C3F29F40E94A41380938A02FE
:1028200008959FE0980F983078F421E030E0A901F6
:1028300002C0440F551F9A95E2F7CA019091860293
:10284000892B8093860208958D3F21F48091840224
:1028500081600BC08E3F21F480918402826005C0AC
:102860008F3F29F4809184028460809384020895CC
:102870008D3E39F49091880297FF35C010928802FE
:1028800059C08E3E29F4909188021916BCF32BC0D2
:10289000909187028F3E29F497FF25C010928702FE
:1028A00049C0803F19F41916CCF31DC090918902DC
:1028B000893F29F41916BCF4109289023BC08A3F63
:1028C00019F497FF10C0F8CF8B3F39F490918A022A
:1028D00097FF09C010928A022DC08C3F21F490917D
:1028E0008A021916BCF39FE0980F983080F421E01B
:1028F00030E0A90102C0440F551F9A95E2F7CA01C2
:1029000080959091860289238093860213C08D3F23
:1029100021F4809184028E7F0BC08E3F21F4809140
:1029200084028D7F05C08F3F29F4809184028B7FC4
:102930008093840280918702811106C08091880271
:10294000811102C01092830280918902811106C018
:1029500080918A02811102C01092820208950E9421
:102960001C2120918702211104C02091880222237A
:1029700021F090938102809380022091890221119D
:1029800004C020918A02222321F090937F02809339
:102990007E0285E892E00C94881FEF92FF920F93DD
:1029A0001F93CF93DF9300D000D000D0CDB7DEB718
:1029B00086E0E5E8F2E0DE01119601900D928A953D
:1029C000E1F7E0908702F09088020091890210916F
:1029D0008A02109287021092880210928902109245
:1029E0008A02E11003C0FF2009F45DC080918002DB
:1029F000909181020E943421AC019091830299232D
:102A000039F020910A0130E02417350758F04BC007
:102A100020910B018AE0289F90011124241735078B
:102A200018F041C09F3F19F09F5F90938302EE2002
:102A300061F00E9465131E1414F09FEF01C091E035
:102A4000989F902D112490938702FF2061F00E949F
:102A500065131F1414F09FEF01C091E0989F902D13
:102A6000112490938802309187023323E1F0209162
:102A700088022223C1F045EB3403C00111249923BD
:102A800019F09093870203C081E08093870235EBB1
:102A90002303C0011124992319F09093880203C0E5
:102AA00081E080938802011103C0112309F45DC005
:102AB00080917E0290917F020E943421AC0190911E
:102AC0008202992339F02091060130E0241735075E
:102AD00058F04BC0209107018AE0289F90011124F3
:102AE0002417350718F041C09F3F19F09F5F90935E
:102AF0008202002361F00E94A413101614F09FEFCD
:102B000001C091E0989F902D112490938902112388
:102B100061F00E94A413111614F09FEF01C091E020
:102B2000989F902D112490938A023091890233232B
:102B3000E1F020918A022223C1F045EB3403C00169
:102B40001124992319F09093890203C081E08093A6
:102B5000890235EB2303C0011124992319F09093C6
:102B60008A0203C081E080938A02809187028111EA
:102B70000BC080918802811107C080918902811168
:102B800003C080918A0281110E94AF14EB82FC8203
:102B90000D831E8386E0FE013196A5E8B2E0019028
:102BA0000D928A95E1F726960FB6F894DEBF0FBE18
:102BB000CDBFDF91CF911F910F91FF90EF900895BE
:102BC000E5E8F2E086E0DF011D928A95E9F71092D0
:102BD000830210928202109284020895EF92FF9273
:102BE0000F931F93CF93DF938B01682F11110AC0AE
:102BF000442329F0E82FF0E0E155FD4F6491762F52
:102C0000862F75C0212F30E0E82FF0E0442321F01B
:102C1000E155FD4FE491F0E046E0049FC00111242E
:102C2000CFEFD0E0BE010E947C284BEA4603C001F2
:102C3000479F900D1124800F911D800F911D982F9B
:102C4000990F890FAE01421B530B4E9FD0014F9F2E
:102C5000B00D5E9FB00D11249B2F189FA001112471
:102C6000452F55278E01041B150B0E9FA0010F9FAA
:102C7000500D1E9F500D11247E01E81AF108E29EAE
:102C80008001E39E100DF29E100D1124212F332799
:102C9000C21BD30BCE9F9001CF9F300DDE9F300D16
:102CA000112462307105A9F048F46115710569F0CD
:102CB00061307105C9F48B2F752F0DC0643071051B
:102CC00081F058F06630710579F47E2F8B2F932FA9
:102CD0000DC0832F7B2F9E2F09C08E2F7B2F952F0A
:102CE00005C08E2F732F02C07E2F852F692FDF9195
:102CF000CF911F910F91FF90EF90089541E00E94B6
:102D0000EE15089508950E947E160895CF93DF93DF
:102D1000762FE901682F842F0E94831679836883B8
:102D20008A83DF91CF9108958091DA02282F26952A
:102D300030E02115310519F48170826005C025321B
:102D4000310524F0817088648093DA02089588E068
:102D500090E00C942B29CF92DF92EF92FF926B01BF
:102D60007C010E949416B701A60188E090E0FF90D4
:102D7000EF90DF90CF900C944929EAEDF2E083E0E8
:102D8000808311828FEF82838383148260817181BB
:102D9000828193810C94AB168091DA0280FF02C08D
:102DA0008695089580E008959091DE02933018F49E
:102DB0009F5F9093DE02882351F06091DA02709158
:102DC000DB028091DC029091DD020C94AB16089539
:102DD00081E00C94D4169091DE02992319F0915061
:102DE0009093DE02882351F06091DA027091DB0249
:102DF0008091DC029091DD020C94AB16089581E085
:102E00000C94EB1670E00C94EF1C60911001809113
:102E1000DA0280FF0AC080910F0123E0829FC00187
:102E2000112481529D4F0C940217809111019091B1
:102E30001201891780F7E82FF0E09F01220F331F5E
:102E4000E20FF31FE152FD4F1182108212828F5F59
:102E5000F0CF9091DA0290FF16C09091110120916D
:102E60001201921770F4E92FF0E0DF01AA0FBB1FE7
:102E7000EA0FFB1FE152FD4F8183608342839F5F16
:102E8000F0CF0C9405170895CF93DF9300D01F92D5
:102E9000CDB7DEB79091DA0290FF0AC09E012F5F96
:102EA0003F4F0E9486164B8169818A810E942917B3
:102EB0000F900F900F90DF91CF910895CF93DF93F4
:102EC000EC01EC81F0E0E655FE4F4491EAEDF2E0D2
:102ED000628181810E9444178C818F5F8C83DF9196
:102EE000CF910895CF93DF93EC01EAEDF2E04381B7
:102EF00062818C810E9444178C818F5F8C83DF916B
:102F0000CF9108950F931F93CF93DF9300D01F921B
:102F1000CDB7DEB78C0180918B0281110AC09E0172
:102F20002F5F3F4F4FEF6FEF0E9486168A8180938D
:102F30008B02F8018481813051F028F0823061F4F5
:102F400040918B020AC080918B0240E007C06091E3
:102F50008B0240E080E003C040E080E060E00E943F
:102F60002917F801848190E0019663E070E00E94E7
:102F7000902884830F900F900F90DF91CF911F9135
:102F80000F910895AF92BF92CF92DF92EF92FF928E
:102F90000F931F93CF93DF9300D01F92CDB7DEB76F
:102FA000182FF62E042FE22E9091DA0290FF6DC0BA
:102FB000E92FE695AE2FB0E0A256BE4F8C918093DC
:102FC00095029E7F923061F49E012F5F3F4F812FCB
:102FD0000E9486164B8169818A810E94291743C00D
:102FE000823019F40091DD023EC0863019F4109150
:102FF000DB0239C08930D9F38931A9F5E9518E2F27
:103000008170D82EE695F0E0E655FD4FA590B4907E
:10301000C12CBB2460911301C61618F52C2D30E08D
:10302000A29EC001A39E900DB29E900D112470E04F
:103030000E947C28812FD11002C0860F01C0861B00
:1030400090911101290F311DA901440F551F240F23
:10305000351F21523D4F402F6F2D0E948616C3947D
:10306000D9CF0E9405171093DB02F092DC02009387
:10307000DD02EE2051F06091DA027091DB02809166
:10308000DC029091DD020E94AB160F900F900F9022
:10309000DF91CF911F910F91FF90EF90DF90CF9034
:1030A000BF90AF900895EAEDF2E09181282F43811F
:1030B000628188E0890F0C94C21781E00C94531848
:1030C000EAEDF2E09181282F4381628188EF890F38
:1030D0000C94C21781E00C946018EAEDF2E0628172
:1030E00028E0620F08F46FEF282F438181810C9450
:1030F000C21781E00C946D18EAEDF2E0628128E0DD
:10310000621B08F460E0282F438181810C94C21770
:1031100081E00C947C18EAEDF2E0438128E0420F54
:1031200008F44FEF282F628181810C94C21781E04F
:103130000C948B18EAEDF2E0438128E0421B08F47E
:1031400040E0282F628181810C94C21781E00C94A9
:103150009A1820E00C94C217FF920F931F93CF93FD
:10316000DF93EC01F12C0FEF10E060911301F616E4
:10317000F0F4809111012F2D30E0280F311DC9018D
:10318000880F991F280F391F21523D4F70E0C80149
:103190000E949028962F8C814091DD026091DC0284
:1031A000F99E800D11240E948616F394DECF0E94B2
:1031B00005179A818C8190FF02C08F5F01C08150FA
:1031C0008C83DF91CF911F910F91FF900895AF9263
:1031D000BF92CF92DF92EF92FF920F931F93CF9304
:1031E000DF93FC01828180FF02C00FEF01C001E08C
:1031F00010E04CE0A42E80911301181708F043C092
:1032000080911101C12ED12CE601C80FD11DCE0134
:10321000880F991FC80FD91FC152DD4F198218821C
:103220001A8234E0E32EF12CB12C80918D028B0DAB
:103230008D302CF06A2D0E946E28892F05C087FFE3
:1032400003C090911301890F082E000C990BC8162A
:10325000D90691F48091DD028E9DA0018F9D500DC5
:10326000112455954795559547959E016091DC022F
:103270008091DB020E948616B00EF1E0EF1AF10891
:10328000A1F61F5FB8CF0E94051780918D02013013
:1032900031F4811102C080911301815007C090E088
:1032A00001966091130170E00E94902880938D0236
:1032B000DF91CF911F910F91FF90EF90DF90CF9012
:1032C000BF90AF900895CF9380911101909112011A
:1032D000891770F4E82FF0E09F01220F331FE20FEF
:1032E000F31FE152FD4F1182108212828F5FF0CFE7
:1032F000C0E060911301C617C0F5EC2FF0E070E05C
:10330000CF010E94902820911101820F20918C0200
:10331000022E000C330B90E0E217F307CCF0209163
:103320000E01022E000C330B2E173F078CF09C0170
:10333000220F331F820F931F9C0121523D4F40915A
:10334000DD026091DC028091DB020E9486160BC0D8
:10335000FC01EE0FFF1F8E0F9F1FFC01E152FD4F7E
:10336000118210821282CF5FC4CF0E940517209174
:103370000D0180918C02820F80938C0290910E013E
:10338000920F90930E0119165CF4082E000C990B05
:103390004091130150E041505109841795071CF0EA
:1033A000219520930D01CF9108958F929F92AF9216
:1033B000BF92CF92DF92EF92FF920F931F93CF9322
:1033C000DF938C01FC014481C42FD0E09E01DE011B
:1033D0000E94D4289B01AC010E94EA286B017C0169
:1033E000E0E2F0E0EC1BFD0BA5E5B0E09B01AC01D9
:1033F0000E94EA284B015C019F01DF010E94CC285A
:103400009B01AC010E94F5289B01AC012C0D3D1DD8
:103410004E1D5F1DC501B4010E94A428C22FD22FEA
:103420002A3228F4F3E02F9F900111240DC025E5E6
:1034300030E02C1B3109C901880F991F280F391F53
:1034400037FF02C02F5F3F4F35952795C22FC0959C
:10345000F12C85E5E82EED1A80911301F816C8F4D9
:10346000F1FC02C08E2D01C08D2F909111012F2DE6
:1034700030E0290F311DA901440F551F240F351FBE
:1034800021523D4F4C2F6091DC020E948616F3942E
:10349000E3CF0E940517F8018481811102C091E0F9
:1034A00003C0803219F49FEF90930C0190910C01AE
:1034B000890FF8018483DF91CF911F910F91FF90C5
:1034C000EF90DF90CF90BF90AF909F908F90089536
:1034D0000F931F93CF93DF93EC0100E010E08091F6
:1034E0001301282F30E00217130724F590911101E2
:1034F0009801290F311DA901440F551F240F351FB5
:1035000021523D4F869590E04C81081719071CF415
:10351000442331F002C0411103C04091DD0201C0DB
:1035200040E06091DC028091DB020E9486160F5F12
:103530001F4FD5CF0E9405178C8190E001968170B6
:1035400099278C83DF91CF911F910F910895EAED18
:10355000F2E080818E7F808360817181828193819E
:103560000E94AB16109296022FEF80E792E0215056
:1035700080409040E1F700C000000C940517609176
:10358000DA02669570E04BE050E084E191E00E9441
:103590000929892B19F481E0809396020E941C214D
:1035A00090938F0280938E0208959091DA0290FF9B
:1035B00035C09170811102C0926006C0853210F052
:1035C000986402C0880F982B9093DA02662351F01A
:1035D0006091DA027091DB028091DC029091DD0251
:1035E0000E94AB166091DA02669570E04BE050E005
:1035F00084E191E00E940929892B19F0109296022A
:1036000002C00E94BF1A81E0809391024091DD02C6
:103610006091DC028091DB020C94A9180895682F58
:103620009091DA02969581E0890F853208F081E069
:103630000C94D51A81E00C940F1B682F9091DA023C
:1036400096958FEF890F09F484E20C94D51A81E0E6
:103650000C941D1B61E00C94D51AEAEDF2E0808118
:103660008160808386950C942A1B8091DA0280FD0C
:103670000C94A71A0C942D1B60E00C94D51A809121
:10368000940281112EC00E94180E811104C00E9464
:10369000C00E0E94BD160E94A7166093DA027093B6
:1036A000DB028093DC029093DD026E7F61F40E9466
:1036B000BD160E94A7166093DA027093DB02809316
:1036C000DC029093DD020E94941610929602809183
:1036D000DA0280FF03C086950E943C1B81E0809344
:1036E000940208950F931F93CF93DF9380919602D6
:1036F000882309F485C080919502E091DA02E6956D
:10370000E81BE0939002823049F4F0E0EA55FE4F66
:10371000E491CE2FD0E00EE517E149C0863049F4A0
:10372000F0E0ED55FE4FE491CE2FD0E002E717E137
:103730003EC0893051F4E695F0E0E056FE4FE4914A
:10374000CE2FD0E00CEA18E132C08F3051F4E6956C
:10375000F0E0E356FE4FE491CE2FD0E007EE18E103
:1037600026C0853149F4F0E0E656FE4FE491CE2FB5
:10377000D0E003E619E11BC0883181F0833239F4CF
:10378000E8E9F1E0C591D49102E817E110C0843274
:1037900051F4C4EFD1E008E61AE109C0C8E2D0E074
:1037A00005ED19E104C0C0EDD7E002E816E1809113
:1037B0009102882361F0109291020E941C21909343
:1037C0008F0280938E0210929302109292020E94B6
:1037D0001C21E0918E02F0918F028E1B9F0B8F3F78
:1037E0009F4770F4EC0FFD1FF0938F02E0938E0261
:1037F0008EE892E0F801DF91CF911F910F9109942B
:10380000DF91CF911F910F910895882311F0FA0154
:1038100001C0FB010994CF93DF93C82FD62F0E94DC
:10382000CC168C1740F00E94CC168D1720F4DF9137
:10383000CF910C941A1B8C2FDF91CF910C942A1BE3
:103840001F93CF93DF93FB0112811111C3C0EC01D1
:103850000E942F0D8272CD3CFCE5DF0709F49AC06F
:10386000A8F5C73CECE5DE0709F476C0A8F4C43C33
:103870009CE5D90709F45FC028F4C33CDC4509F492
:1038800057C054C0C53C9CE5D90709F459C0C63C93
:10389000DC4509F45CC04AC0CA3CFCE5DF0709F41A
:1038A0006AC050F4C83CECE5DE0709F45AC0C93CD4
:1038B000DC4509F45BC03AC0CB3C9CE5D90709F470
:1038C0005FC0CC3CDC4509F460C030C0C23DFCE5C3
:1038D000DF0709F46FC088F4CF3C9CE5D90709F4F1
:1038E00060C008F45CC0C03DFCE5DF0709F45CC0C3
:1038F000C13DDC4509F45BC019C0C53D9CE5D90755
:1039000009F460C050F4C33DFCE5DF0709F455C07D
:10391000C43DDC4509F454C009C0C63D9CE5D90747
:1039200009F455C0CE35DD4509F454C011E052C04C
:103930000E94351B4FC047E25BE16AE17BE104C0B6
:103940004AE15BE167E27BE10E94051C43C04AE675
:1039500058E16DE578E1F8CF4DE558E16AE678E1A8
:10396000F3CF48E858E169E778E1EECF49E758E15D
:1039700068E878E1E9CF46EA58E167E978E1E4CF21
:1039800047E958E166EA78E1DFCF4FEF56E168EEAC
:1039900076E1DACF48EE56E16FEF76E1D5CF81E000
:1039A00017C065E082E010C068E086E00DC06EE000
:1039B00089E00AC064E18FE007C067E185E104C0E7
:1039C00088E106C062E289E10E940B1C03C083E229
:1039D0000E942A1B812FDF91CF911F910895569A43
:1039E0002BB12F7B3BB130644FB7F894FC01CB0176
:1039F000880F991F680F791F6E0F7F1FE617F70753
:103A000089F0819198E03BB9000000C087FF2BB995
:103A1000880F000000C000C000C02BB900C09A95FC
:103A200091F7ECCF4FBF8FE594E00197F1F700C01D
:103A300000000895CF93DF93EC01FB01828188237E
:103A400009F43CC1C430FDE5DF0760F4CB3F9CE5E1
:103A5000D90788F49E0122503C452431310508F0F5
:103A60002EC109C0C236EDE5DE0729F0C63AFDE5F4
:103A7000DF0709F024C10E942B0E9093C9028093A6
:103A8000C802C1318CE5D80709F4C6C008F042C0AD
:103A9000C930ECE5DE0709F49BC000F5C5308CE5C4
:103AA000D80709F485C078F4C330ECE5DE0709F4E3
:103AB00078C008F07AC0C230DC4509F0F5C08091CA
:103AC000C8028160EFC0C7309CE5D90709F478C00F
:103AD00008F07AC08091C8028061E4C0CD30FCE576
:103AE000DF0709F487C058F4CB309CE5D90709F407
:103AF00079C008F07BC08091C80288606FC0CF3069
:103B0000FCE5DF0709F480C008F082C08091C8029C
:103B1000877FC8C0CE3F9CE5D90709F471C000F586
:103B2000C531FCE5DF0709F485C068F4C3319CE5C5
:103B3000D90709F475C008F095C00E94DC07809190
:103B4000C8028F77AFC0CC3FFCE5DF07A9F108F0D2
:103B500054C0CB3FDC4509F0A7C08091C90240C0EA
:103B6000C230EDE5DE0709F489C058F4C1158DE5D2
:103B7000D80709F45AC008F069C08091C902826070
:103B80002FC0C236EDE5DE0709F47CC0C63AFDE57C
:103B9000DF0709F481C0C330DD4509F085C080E04E
:103BA0006EC08091C80282607DC08091C80216C03C
:103BB0008091C802886076C08091C90282604FC03F
:103BC0008091C80280626EC08091C80280646AC021
:103BD0000E94DC078091C802806864C0846062C073
:103BE00081603DC08091C8028E7F5CC08091C80218
:103BF0008D7F58C08091C80216C08091C90218C03C
:103C00008091C9028D7F2BC08091C8028F7E4AC0EF
:103C10008091C8028F7D46C08091C8028F7B42C0D0
:103C20008091C802877F8B7F3DC08091C9028D7FC4
:103C30008E7F15C08091C80282FB222720F991E077
:103C4000922790FB82F990FB83F92CC08091C902E6
:103C5000982F909591708E7F892B90FB81F980939E
:103C6000C90222C00E94DC078091C80287FB22277C
:103C700020F991E0922790FB87F914C081E00E941F
:103C8000C20E12C08091C80284FB222720F991E065
:103C9000922790FB84F906C08091C802982F9095D6
:103CA00090FB80F98093C8028091C8029091C9026C
:103CB0000E943C0E0E94DC0780E001C081E0DF91A1
:103CC000CF910895CF93DF9386319C4541F5EB0169
:103CD0000E942F0D982F8A812091020130910301BB
:103CE000882379F09A7A81E009F480E08093970242
:103CF000911102C069E201C065E3C9010E94582028
:103D00000AC080919702811102C069E201C065E397
:103D1000C9010E9463200E94710D80E001C081E012
:103D2000DF91CF9108950F931F93CF93DF93C42F0B
:103D3000D22FFC0182818823C9F040939A020E940D
:103D40001C21909399028093980280E28C0F883016
:103D500008F057C0C77081E001C0880FCA95EAF724
:103D6000DF91CF911F910F910C94390580919A02A8
:103D7000481330C080919802909199020E9434219A
:103D8000883C910538F510E21D0FCD17B9F080E29F
:103D90008C0F883040F4C77081E001C0880FCA954D
:103DA000EAF70E944005183028F581E09D2F9770B2
:103DB00001C0880F9A95EAF70E943905802F0E946A
:103DC00030051830F0F4D77081E001C0880FDA9523
:103DD000EAF70AC080E28C0F883098F4C77081E05F
:103DE00001C0880FCA95EAF7DF91CF911F910F911B
:103DF0000C944005802FDF91CF911F910F910C946F
:103E00003005DF91CF911F910F9108950F939C0181
:103E1000CB01243F4CE5340731F188F4293DFCE522
:103E20003F07D9F02A3D4CE5340779F1283D3C4560
:103E3000A9F506E221EE41EE68ED7CE52BC0263FB8
:103E4000FCE53F07E1F0A8F0273F3C4539F507E2E4
:103E500025EE46EE67EF7CE51DC007E225EE45EE58
:103E600069ED7CE517C006E221EE40EE64EF7CE5EB
:103E700011C007E225EE44EE65EF7CE50BC006E2DB
:103E800021EE42EE66EF7CE505C008E221E045EE5A
:103E90006AED7CE50E94931E80E008C0FC018281EF
:103EA000882319F010929A0201C081E00F910895C1
:103EB0009093C5018093C40108959093A0028093CC
:103EC0009F020895E0919F02F091A002309721F0A7
:103ED0000190F081E02D099480E00895E0919F0227
:103EE000F091A002309799F020912B01222359F0F4
:103EF0002091C80227FF07C0DC012C9111962C935A
:103F0000119726E02C930280F381E02D0994089507
:103F1000E0919F02F091A002309739F022E0DC019D
:103F20002C930480F581E02D0994089520919D0241
:103F300030919E022817390771F090939E0280936A
:103F40009D02E0919F02F091A002309721F006803F
:103F5000F781E02D0994089520919B0230919C02F5
:103F60002817390771F090939C0280939B02E0918F
:103F70009F02F091A002309721F00084F185E02D9E
:103F800009940895FC01329680912B01882331F029
:103F90008091C80287FF02C09EE101C096E080E0E8
:103FA000915028F021912223D9F38F5FF9CF089502
:103FB000662351F120912B012223E9F02091C802C0
:103FC00027FF19C0462F4695469546954E31E0F499
:103FD000677021E030E002C0220F331F6A95E2F7DC
:103FE000FC01E40FF11D828190E02823392381E058
:103FF000232B69F409C0FC013296089621916217BF
:1040000029F0E817F907D1F780E0089581E00895D5
:104010009C01FC0132969FEF80E04191461789F0A8
:104020009F3F19F4411101C0982F8F5F8630A9F787
:104030009F3F39F0F901E90FF11D97FDFA95628371
:10404000089508959C012A5F3F4FFC014281461369
:1040500001C01282019682179307B9F70895262F9F
:104060002695269526952E3168F4FC01E20FF11D68
:10407000677021E030E001C0220F6A95EAF7828183
:10408000282B22830895262F2695269526952E31B6
:1040900070F4FC01E20FF11D677021E030E001C017
:1040A000220F6A95EAF720958281282322830895BA
:1040B00020912B01222329F02091C80227FD0C9486
:1040C0002F200C94082020912B01222329F02091ED
:1040D000C80227FD0C9443200C94222020912B0130
:1040E000FC013296222331F08091C80287FF02C082
:1040F0008EE101C086E0DF011D928A95E9F70895FF
:1041000008950C94802083E08093A1020C94812078
:10411000811102C081E001C082E08093A1020C9471
:1041200081200C94882081E08093A1020C9481204E
:104130000C94932008950C949A200C949B200C943A
:104140009A200C949A200C949A20CF930E94A1203C
:104150000E94C6120E949F20C0E08C2F0E94F01186
:10416000892B29F4CF5FC430C1F780E001C081E022
:10417000CF91089508951F920F920FB60F921124B8
:104180008F939F93AF93BF938091A202811113C02D
:104190008091030390910403A0910503B09106035D
:1041A0004196A11DB11D8093030390930403A09336
:1041B0000503B0930603BF91AF919F918F910F902C
:1041C0000FBE0F901F90189580910B03843031F132
:1041D0000E948C031092A20220E488E190E00FB6C6
:1041E000F894A895809360000FBE2093600083B779
:1041F000817F846083BF83B7816083BF7894889513
:1042000083B78E7F83BF0FB6F894A8958091600026
:10421000886180936000109260000FBE08950E9434
:10422000DC070C94900382E084BD93E095BD9AEF87
:1042300097BD80936E0008952FB7F8948091030383
:1042400090910403A0910503B09106032FBF089538
:104250002FB7F894609103037091040380910503D4
:10426000909106032FBF08959C014FB7F894809159
:10427000030390910403A0910503B09106034FBF7F
:10428000821B930B089578941F920F920FB60F9292
:1042900011248F939F93AF93BF93809103039091C9
:1042A0000403A0910503B09106030196A11DB11D61
:1042B0008093030390930403A0930503B093060334
:1042C000BF91AF919F918F910F900FBE0F901F9054
:1042D000189581E08093E00080E28093D8001092EE
:1042E000C9008FE19EE40197F1F700C0000087E06C
:1042F00090EBDC018093140390931503A0931603B5
:10430000B09317039CE088E10FB6F894A8958093CA
:1043100060000FBE90936000FFCF8091C6020895A9
:10432000089522E02093E9002FEF3091E80021501A
:1043300035FD06C035ED3A95F1F700002111F5CFB6
:104340002091E80025FF0BC040E050E066E070E0FF
:104350000E94D0238091E8008E778093E800089532
:10436000CF93DF9320912B01222339F02091C802B3
:1043700027FF03C060E222E002C068E021E0209352
:10438000E9002FEF3091E800215035FD06C035EDF2
:104390003A95F1F700002111F5CF2091E80025FFB3
:1043A0001DC0EC0180912B01811105C040E050E05F
:1043B00068E070E003C070E040E050E0CE010E9491
:1043C000D0238091E8008E778093E80080E2FE01A0
:1043D000A6EAB2E001900D928A95E1F7DF91CF91C4
:1043E00008958093A3027093A5026093A402809124
:1043F0000B03843001F582E08093E9008FEF909108
:10440000E800815095FD06C095ED9A95F1F7000002
:104410008111F5CF8091E80085FF0DC040E050E0AC
:1044200063E070E083EA92E00E94D0238091E8008C
:104430008E778093E8000895BC0184E00C94F1210C
:10444000BC0183E00C94F12180910A03811109C021
:104450000E9461250E94BE258091E20084608093C5
:10446000E200089510920A0308950C949820609138
:10447000070381E0611101C080E00C9483209091DA
:104480000B0381E0943009F080E0609107030C9405
:10449000882042E061EC81E00E94DA2442E261EC93
:1044A00082E00E94DA2490910B0381E0943009F0BD
:1044B00080E0609107030C94912080910D0383307C
:1044C00009F461C030F4813071F0823009F49AC08F
:1044D00008958A3009F486C08B3009F46CC08930A5
:1044E00009F0A8C020C080910C03813A09F0A2C055
:1044F0008091E800877F8093E8008091100390917D
:104500001103892B21F460E286EA92E003C060E0A7
:1045100080E090E070E00E941B248091E8008B779F
:104520008093E800089580910C03813209F082C0E5
:104530008091100390911103029708F07BC0809145
:10454000E800877F8093E8008091E80082FD05C045
:1045500080910B038111F8CF6DC02091F300809101
:10456000F20090E0922B029731F48091F1008130BB
:1045700011F0863021F48091F1008093C602809181
:10458000E8008B7753C080910C03813A09F052C048
:104590008091100390911103892B09F04BC08091F9
:1045A000E800877F8093E8008091E80080FFFCCFDF
:1045B00080912B0136C080910C038132D9F5809116
:1045C000100390911103892BA9F58091E800877F52
:1045D0008093E8000E940F2580910E0380932B01A9
:1045E0000C94DC0780910C03813221F58091E80066
:1045F000877F8093E8000E940F2580910F038093AE
:10460000C702089580910C03813AA1F48091E800DB
:10461000877F8093E8008091E80080FFFCCF809145
:10462000C7028093F1008091E8008E778093E800C4
:104630000C940F25089584B7877F84BF0FB6F89434
:10464000A89580916000886180936000109260005E
:104650000FBE90E080E80FB6F894809361009093CD
:1046600061000FBE0C9493200E9461250E94BE251C
:10467000E2EEF0E080818460808378940C9453288B
:104680008FE191E00C945D1F80910B038530A9F4BC
:1046900080910B03853079F40E94E4208091090316
:1046A0008823B1F30E94A520882391F30E94BA23A6
:1046B0000E94DC07EDCF0C940F21089508950C940F
:1046C0006123292F332723303105C9F060F42130CD
:1046D000310581F02230310509F044C08BE390E0D0
:1046E00023EE33E043C021323105E1F022323105BF
:1046F00049F138C082E190E02EE134E037C09927DB
:104700008130910549F028F0029761F5EFEAF3E076
:1047100005C0EFEDF3E002C0EDEBF3E0849190E033
:104720009F0124C06115710541F061307105D1F41C
:1047300089E090E02EE034E019C089E090E025EFB8
:1047400033E014C06115710541F06130710551F419
:1047500086EB90E020E334E009C080E490E026EEB0
:1047600034E004C080E090E020E030E0FA013183E2
:104770002083089580E189BD82E189BD09B400FEEE
:10478000FDCF8091D8008F7D8093D8008091E0008C
:1047900082608093E0008091E00081FDFCCF08956D
:1047A000CF92DF92EF92FF920F931F93CF93DF93FD
:1047B000EC018B017A010E942E25811133C0E11496
:1047C000F10439F0F70180819181081B190BC80FA2
:1047D000D91FC12CD12C0115110519F18091E800C8
:1047E00085FD16C08091E8008E778093E800E11483
:1047F000F10449F0F70180819181C80ED91ED18260
:10480000C08285E00FC00E942E25882321F30AC0B4
:1048100089918093F10001501109FFEFCF1ADF0A4F
:10482000DACF80E0DF91CF911F910F91FF90EF9051
:10483000DF90CF9008952091120330911303261733
:10484000370748F06115710539F42091E8002E779B
:104850002093E80001C0B901FC0120E06115710559
:1048600079F180910B038823F1F18530F1F180918A
:10487000E80083FD3CC08091E80082FD2EC080915D
:10488000E80080FFEBCF2091F3008091F20090E0F0
:10489000922B6115710551F08830910538F4219102
:1048A0002093F100615071090196F3CF21E0089740
:1048B00009F020E08091E8008E778093E800CECF69
:1048C0002111CFCF0AC080910B03882361F085307E
:1048D00061F08091E80083FD0AC08091E80082FFCA
:1048E000F2CF80E0089582E0089583E0089581E0AA
:1048F000089520911203309113032617370748F0CB
:104900006115710539F42091E8002E772093E800B5
:1049100001C0B901FC0120E06115710591F18091A0
:104920000B03882309F440C0853009F43FC080910F
:10493000E80083FD3DC08091E80082FD2FC080919A
:10494000E80080FFE9CF2091F3008091F20090E031
:10495000922B6115710559F08830910540F424912E
:104960002093F1003196615071090196F2CF21E058
:10497000089709F020E08091E8008E778093E800A6
:10498000CBCF2111CCCF0AC080910B03882361F0DB
:10499000853061F08091E80083FD0AC08091E800D5
:1049A00082FFF2CF80E0089582E0089583E00895C9
:1049B00081E00895982F973068F59093E900981753
:1049C00039F07091EC002091ED005091F00003C09F
:1049D000242F762F50E021FD02C09F5FECCF309155
:1049E000EB003E7F3093EB003091ED003D7F309344
:1049F000ED003091EB0031603093EB007093EC00F0
:104A00002093ED005093F0002091EE0027FDE5CFBC
:104A100080E008958F708093E90081E0089580918F
:104A20000C0387FF11C08091E80082FD05C08091D2
:104A30000B038111F8CF11C08091E8008B770BC078
:104A400080910B03882349F08091E80080FFF8CF24
:104A50008091E8008E778093E80008952091E4002B
:104A60003091E50095E64091EC00842F817040FF85
:104A700023C08091E80080FD1DC080910B03882336
:104A800099F0853099F08091EB0085FD11C040913F
:104A9000E4005091E5002417350729F3915011F0F7
:104AA0009A01E1CF84E0089582E0089583E00895BB
:104AB00081E0089580E008954091E80042FFDDCF55
:104AC00008950E94CF250E94D725E0EEF0E0808176
:104AD00081608083E8EDF0E080818F77808319BC6E
:104AE000A7EDB0E08C918E7F8C9380818F7E808348
:104AF00010920A0308950F931F93CF93DF930E94A0
:104B0000CF250E94D725C8EDD0E088818F77888394
:104B100088818068888388818F7D888319BC109202
:104B20000B0310920703109209031092080300EE82
:104B300010E0F80180818B7F808388818160888389
:104B400042E060E080E00E94DA24E1EEF0E0808163
:104B50008E7F8083E2EEF0E08081816080838081BF
:104B600088608083F80180818E7F80838881806166
:104B70008883DF91CF911F910F910895E8EDF0E0C8
:104B800080818F7E8083E7EDF0E08081816080838B
:104B900084E082BF81E080930A030C947B25E8EDDA
:104BA000F0E080818E7F80831092E2000895109261
:104BB000DA001092E10008951F920F920FB60F9243
:104BC00011242F933F934F935F936F937F938F9312
:104BD0009F93AF93BF93EF93FF938091E10082FF88
:104BE0000BC08091E20082FF07C08091E1008B7FC3
:104BF0008093E1000E9452288091DA0080FF1FC05C
:104C00008091D80080FF1BC08091DA008E7F809356
:104C1000DA008091D90080FF0DC080E189BD82E17A
:104C200089BD09B400FEFDCF81E080930B030E9493
:104C3000242205C019BC10920B030E9432228091DD
:104C4000E10080FF19C08091E20080FF15C08091D3
:104C5000E2008E7F8093E2008091E2008061809389
:104C6000E2008091D80080628093D80019BC85E072
:104C700080930B030E9437228091E10084FF30C0B3
:104C80008091E20084FF2CC080E189BD82E189BD72
:104C900009B400FEFDCF8091D8008F7D8093D800AD
:104CA0008091E1008F7E8093E1008091E2008F7E11
:104CB0008093E2008091E20081608093E200809125
:104CC0000703882311F084E007C08091E30087FD8B
:104CD00002C081E001C083E080930B030E943F2269
:104CE0008091E10083FF29C08091E20083FF25C00D
:104CF0008091E100877F8093E10082E080930B0345
:104D0000109207038091E1008E7F8093E1008091F3
:104D1000E2008E7F8093E2008091E20080618093C8
:104D2000E20042E060E080E00E94DA248091F0003E
:104D300088608093F0000E943522FF91EF91BF912F
:104D4000AF919F918F917F916F915F914F913F9123
:104D50002F910F900FBE0F901F9018951F920F92DA
:104D60000FB60F9211242F933F934F935F936F933E
:104D70007F938F939F93AF93BF93CF93DF93EF93E3
:104D8000FF93C091E900CF708091EC00D82FD170D3
:104D900080FDD0E81092E9008091F000877F809339
:104DA000F00078940E94F2261092E9008091F000C1
:104DB00088608093F000CD2BCF70C093E900FF9105
:104DC000EF91DF91CF91BF91AF919F918F917F91A3
:104DD0006F915F914F913F912F910F900FBE0F9068
:104DE0001F9018951F93CF93DF93CDB7DEB7AA9787
:104DF0000FB6F894DEBF0FBECDBFECE0F3E08091BC
:104E0000F100819323E0E431F207C9F70E945D22AB
:104E10008091E80083FF2EC180910C0390910D03D7
:104E2000492F50E04A30510508F024C1FA01EE59EB
:104E3000FF4F0C94C628803821F0823809F01AC13F
:104E400008C08091080390910903992389F082603A
:104E50000FC0809110038F70873008F00BC18093D2
:104E6000E9008091EB0085FB882780F91092E9002A
:104E70009091E800977F9093E8008093F100109262
:104E8000F100D1C0282F2D7F09F0F4C0882319F03C
:104E9000823061F0EFC080910E03813009F0EAC0EA
:104EA000933009F080E0809309032EC080910E03B7
:104EB00081112AC0809110038F702FEF280F2630A8
:104EC00008F0D8C08093E9002091EB0020FF1CC0BF
:104ED000933021F48091EB00806214C09091EB003C
:104EE00090619093EB0021E030E0A90102C0440FF3
:104EF000551F8A95E2F74093EA001092EA008091EC
:104F0000EB0088608093EB001092E9008091E8004C
:104F1000877F8093E8000E940F25ACC08111AAC052
:104F200010910E031F778091E3008078812B80938E
:104F3000E3008091E800877F8093E8000E940F25BE
:104F40008091E80080FFFCCF8091E300806880932F
:104F5000E300111102C082E001C083E080930B03E3
:104F600089C08058823008F085C080910E039091EE
:104F70000F038C3D53E0950779F583E08A838AE23D
:104F800089834FB7F894DE01139620E03EE051E2AA
:104F9000E32FF0E050935700E49120FF03C0E29527
:104FA000EF703F5FEF708E2F90E0EA3010F0C79601
:104FB00001C0C0968D939D932F5F243149F74FBF59
:104FC0008091E800877F8093E8006AE270E0CE017C
:104FD00001960E941B2416C060911003709111036A
:104FE000AE014F5F5F4F0E945F23BC01892B09F424
:104FF00041C09091E800977F9093E80089819A8161
:105000000E9479248091E8008B778093E80032C079
:10501000803881F58091E800877F8093E800809157
:1050200007038093F1008091E8008E7772CF8111A1
:1050300021C080910E0390910F0399270297D4F419
:105040008091E800877F8093E80080910E03809331
:1050500007030E940F2580910703811106C08091EC
:10506000E30087FD02C081E001C084E080930B0370
:105070000E9449228091E80083FF0AC08091E800E5
:10508000877F8093E8008091EB0080628093EB0043
:10509000AA960FB6F894DEBF0FBECDBFDF91CF91B9
:1050A0001F9108950895CF9380910B038823A1F059
:1050B000C091E900CF709091EC00892F817090FD34
:1050C00080E8C82B1092E9008091E80083FD0E94DF
:1050D000F226CF70C093E900CF91089587FB082E88
:1050E000062687FD819567FD61950E94FD280EF4D7
:1050F000919507FC81950895AA1BBB1B51E107C040
:10510000AA1FBB1FA617B70710F0A61BB70B881F57
:10511000991F5A95A9F780959095BC01CD010895E6
:1051200097FB072E16F4009407D077FD09D00E9454
:105130007C2807FC05D03EF4909581959F4F0895FB
:10514000709561957F4F0895A1E21A2EAA1BBB1B93
:10515000FD010DC0AA1FBB1FEE1FFF1FA217B30743
:10516000E407F50720F0A21BB30BE40BF50B661F59
:10517000771F881F991F1A9469F76095709580951D
:1051800090959B01AC01BD01CF010895EE0FFF1F6B
:105190000590F491E02D09940E94D428332312F451
:1051A0008A1B9B0B0C94E528A29FB001B39FC00102
:1051B000A39F700D811D1124911DB29F700D811D43
:1051C0001124911D08950E94D428B7FF0895821BD1
:1051D000930B08950E94D428A59F900DB49F900D25
:1051E000A49F800D911D11240895B7FF0C94EA2807
:1051F0000E94EA28821B930B0895991B79E004C052
:10520000991F961708F0961B881F7A95C9F7809505
:105210000895FC014150504030F001900616D1F73E
:105220003197CF010895882799270895FB01DC0164
:1052300004C08D910190801921F441505040C8F76D
:10524000881B990B0895F999FECF92BD81BDF89AFC
:10525000992780B50895A6E1B0E044E050E00C94B1
:105260005D29A8E1B0E042E050E00C945D29262FD2
:10527000F999FECF92BD81BDF89A019700B402164C
:1052800039F01FBA20BD0FB6F894FA9AF99A0FBEFA
:1052900008950396272F0E9438290E943729252F29
:1052A0000E943829242F0C9438290196272F0E9418
:1052B00038290C943729DC01CB01FC01F999FECF88
:1052C00006C0F2BDE1BDF89A319600B40D9241508E
:0A52D0005040B8F70895F894FFCF9E
:1052DA00C8004802280850011E0A140101010200F0
:1052EA000C000C0C01191A1B1C1D1E1F2021228DDB
:1052FA0021B021912120221C22902101E200E90003
:10530A00EA00B500B600B700CD008301CC008A01DF
:10531A009201940121022302240225022602270275
:10532A002A02B300B4006F007000818283E200E9B0
:10533A0000EA00B500B600B700CD008301CC008AB0
:10534A000192019401210223022402250226022746
:10535A00022A02B300B4006F007000818283F0F168
:10536A00F4F5F6F737919293333230319495000180
:10537A00020202020606060909090909090F0F0FA6
:10538A000F0F0F15151518191919191919191919AE
:04539A0019232400AF
:00000001FF
